:100000000C94DC010C94FB010C94FB010C94FB019F
:100010000C94FB010C94FB010C94FB010C94FB0170
:100020000C94FB010C94FB010C94DC1A0C94B21B95
:100030000C94CE150C94FB010C94FB010C94FB0169
:100040000C94FB010C94FB010C94FB010C94FB0140
:100050000C94FB010C9456160C94FB010C94FB01C0
:100060000C94FB010C94FB010C94FB010C94FB0120
:100070000C94FB010C94FB010C94FB010C94FB0110
:100080000C94FB010C94FB010C94FB010C94FB0100
:100090000C94FB010C94FB019A049A04C604C60458
:1000A0002E055906590659064C05E505F605F605CF
:1000B000231C4A1C421D4A1C421D961CB91C421D91
:1000C000101D1F1D2C002C0016000600150004003A
:1000D000050005000F0008001300040007002C00B5
:1000E0002C002C002C001600060015000400050052
:1000F00005000F0008001300040007002C002C006E
:100100002C002C0016000600150004000500050058
:100110000F0008001300040007002C002C002C0026
:100120002C001600060015000400050005000F0055
:1001300008001300040007002C002C002C002C00E9
:100140001600060015000400050005000F00080059
:100150001300040007002C002C002C002C001600BB
:10016000060015000400050005000F00080013003C
:10017000040007002C002C002C002C0016000600A8
:1001800015000400050005000F000800130004001E
:1001900007002C002C002C002C0016000600150077
:1001A0000400050005000F0008001300040007000C
:1001B0002C002C002C002C0016000600150004005A
:1001C000050005000F0008001300040007002C00C4
:1001D0002C002C002C001600060015000400050061
:1001E00005000F0008001300040007002C002C007D
:1001F0002C002C0016000600150004000500050068
:100200000F0008001300040007002C002C002C0035
:100210002C001600060015000400050005000F0064
:1002200008001300040007002C002C002C002C00F8
:100230001600060015000400050005000F00080068
:100240001300040007002C002C002C002C001600CA
:10025000060015000400050005000F00080013004B
:10026000040007002C002C002C002C0016000600B7
:1002700015000400050005000F000800130004002D
:1002800007002C002C00180353006300720061006B
:10029000620062006C0065005000610064000000B4
:1002A000180344006F006E00750074004300610085
:1002B00062006C0065007300000004030904090279
:1002C0003B00020100A0FA09040000010301010043
:1002D00009211101000122400007058103080001E6
:1002E000090401000103000000092111010001229D
:1002F0006D000705820320000112010002000000CA
:10030000084344D72100010102000105010980A131
:1003100001850319012AB700150126B7009501755B
:10032000108100C0050C0901A101850419012AA052
:1003300002150126A002950175108100C005010972
:1003400006A1018506050719E029E7150025019595
:1003500008750181020507190029EF15002501958F
:10036000F0750181020508190129059505750191AE
:1003700002950175039101C005010906A101050758
:1003800019E029E7150025019508750181029501FD
:10039000750881010507190029FF150026FF009542
:1003A0000675088100050819012905950575019153
:1003B00002950175039101C011241FBECFEFD0E259
:1003C000DEBFCDBF11E0A0E0B1E0E0EAFBE300E07A
:1003D0000BBF02C007900D92A239B107D9F723E0F5
:1003E000A2E9B1E001C01D92A535B207E1F70E9474
:1003F0002E120C94CE1D0C94000081E0089581E033
:1004000008950C94FF0108950C9403021F93CF9359
:10041000DF9300D000D01F92CDB7DEB749835A8357
:100420006B833091950189819A81311114C06623C3
:1004300059F0222349F00E949208182F682F8981D1
:100440009A810E943B0803C00E946608182F6981A8
:100450007A81812F04C00E94920869817A810F906D
:100460000F900F900F900F90DF91CF911F910C94F0
:10047000B00FFC01262F40815181628173818481FC
:100480000C94060281E00895CF93DF93EC0160E0C5
:100490000E943902BE01DF91CF910C9404020C94AA
:1004A000DF100C94DB1008950E94E5060E945302B1
:1004B0002FEF84E39CE0215080409040E1F700C0A2
:1004C00000000C947C160F931F93CF93DF938C0145
:1004D00061E00E943902EC01B8010E940102882308
:1004E000F1F1B801CE010E9427148823C1F1B801AF
:1004F000CE010E943B12882391F1B801CE010E94E7
:100500008313882361F1F8018281882309F1CB35B7
:100510008DE5D807C1F050F4C115FCE5DF0781F087
:10052000CF3DDC45A9F40E94C30D19C0CC35EDE5E3
:10053000DE0761F0CD35DD4559F40E940C0D08C091
:100540000E9454020CC00E94150D02C00E94180D9A
:10055000C801DF91CF911F910F910C94FD0180E0B4
:10056000DF91CF911F910F9108950E94B0150C94C7
:10057000CE020E94D1020C94B61508950C94BD02CF
:1005800081E008950C94C0020895CF93C82F0E9473
:10059000BE028C2F0E94C202CF91089580E00C947D
:1005A000C5020E9483140C94C5020E94831490918A
:1005B0009401891721F0809394010C94C502089549
:1005C000CF93DF93CDB7DEB72B970FB6F894DEBF8E
:1005D0000FBECDBF4F83588769877A878B8761119C
:1005E0000E94580C9E012F5F3F4F86E0F901119247
:1005F0008A95E9F785E0FE013796D90101900D92C1
:100600008A95E1F789819A814C815D81452B31F092
:100610009F3F31F491E08F3F19F403C091E001C096
:1006200090E090FF09C049815A816B817C818D8166
:100630009E810E94790B05C0C9010E94420281116E
:10064000F2CF2B960FB6F894DEBF0FBECDBFDF9171
:10065000CF910895FC01808191810E94D408089572
:10066000CF93882309F49CC0C82F8238C1F40E941C
:10067000831481FD95C069E380910201909103018B
:100680000E946B150E947A0C2FEF81EE94E02150AE
:1006900080409040E1F700C0000069E319C0833852
:1006A00001F50E94831480FD7BC063E58091020107
:1006B000909103010E946B150E947A0C2FEF81EE3E
:1006C00094E0215080409040E1F700C0000063E5D5
:1006D00080910201909103010E947615CF910C94B4
:1006E0007A0C8438C1F40E94831482FD59C067E4F7
:1006F00080910201909103010E946B150E947A0C77
:100700002FEF81EE94E0215080409040E1F700C04F
:10071000000067E4DDCF8CEF8C0F813AD0F46C2FB2
:1007200080910201909103010E94EB14882349F00B
:100730006C2F80910201909103010E9476150E9416
:100740007A0C6C2F80910201909103010E946B152D
:10075000C5CF80E28C0F883048F4C77081E001C0BB
:10076000880FCA95EAF70E943B0CB8CFEBE5EC0F77
:10077000E33040F4F0E0E15CFE4F808190E0CF9107
:100780000C94A914C85AC73158F4EC2FF0E0EE0FBE
:10079000FF1FEF5EFE4F80819181CF910C94BF14BB
:1007A000CF910895882309F45BC0682F823879F4CB
:1007B0000E94831481FF54C069E3809102019091EB
:1007C00003010E946B150E947A0C69E310C0833804
:1007D000B1F40E94831480FF43C063E5809102015D
:1007E000909103010E946B150E947A0C63E5809141
:1007F0000201909103010E9476150C947A0C8438C2
:1008000079F40E94831482FF2BC067E48091020177
:10081000909103010E946B150E947A0C67E4E7CF68
:100820008CEF860F813A18F380E2860F883048F407
:10083000677081E001C0880F6A95EAF70E94410C59
:10084000DCCF8BE5860F833020F480E090E00C94C1
:10085000A914685A673120F480E090E00C94BF142A
:1008600008951F93CF93DF93182FEB010E9430035D
:10087000209741F08FE99FE00197F1F700C0000059
:100880002197F6CF812FDF91CF911F910C94D20346
:10089000893319F060E070E002C060E570E00C940C
:1008A0003104882321F00E943B0C0C947A0C0895AB
:1008B000882321F00E94410C0C947A0C0895CF9269
:1008C000DF92EF92FF920F931F93CF93DF937C0100
:1008D000D62FC72FFC011281058102950F700E944F
:1008E000310C8823B9F01123A9F08C2F807F80343C
:1008F00021F080E28D0F883068F08091070382FD3F
:1009000009C082E00E94DA0C0E94310C91E0D82EDE
:10091000D92601C0D12CCC2EC2948FE0C8228C2DB8
:1009200090E08C30910508F0C4C1FC01E45BFF4FFE
:100930000C94761D8C2F807FCF70882311F0C29588
:10094000C07F112399F0CC2309F49FC180E28D0F61
:10095000883010F0D11104C08C2F0E943B0C03C0D2
:100960008C2F0E944B0C0E947A0C8FC18D2F0E94FD
:10097000D203CC2309F49DC180E28D0F883038F179
:10098000DD2329F18C2F0E94510C24C08C2F807FF5
:10099000CF70803211F0C295C07FDD2319F0D130C5
:1009A000A1F13DC08091070382FF17C0112349F0D8
:1009B000CC2329F08C2F0E943B0C0E947A0C80E003
:1009C00065C180E00E94D203CC2309F472C18C2F50
:1009D0000E94410C0E947A0C6CC1112371F000231B
:1009E00041F0013031F40E945B0C8C2B0E94630CAF
:1009F00060C10E945B0C8C2B1DC0002319F00130DC
:100A000009F457C10E94700C25C0112321F0063053
:100A100008F04FC10EC0053008F04BC11BC01123B8
:100A200061F0002331F0F701858180FF2EC18F70C6
:100A300085838C2F0E9451043CC1002359F0D93387
:100A400009F034C1FFEF07EE13E0F1500040104011
:100A5000E1F72AC18C2F0E9458042BC18C2F869558
:100A60008695837019F0813061F023C1112321F044
:100A70008D2F9C2F937002C080E090E00E94A914FB
:100A800020C1112321F08D2F9C2F937002C080E094
:100A900090E00E94BF1415C18C2F837009F047C0ED
:100AA00011110BC12D2F229526952770220F220F91
:100AB0006D2F6F70862F90E0A0E0B0E0022E04C092
:100AC000880F991FAA1FBB1F0A94D2F7D4FF10C02A
:100AD0004FE050E060E070E004C0440F551F661F17
:100AE000771F2A95D2F7409550956095709503C071
:100AF00040E050E0BA01C695C695C3708A019B01DB
:100B0000082B192B2A2B3B2BC901B801C23049F005
:100B100058F4C13019F00E945107CFC00E943F071E
:100B2000CCC00E946307C9C00E943D07C6C0112304
:100B300019F08C2F817001C08695882309F4BDC0FF
:100B40002D2F229526952770220F220F6D2F6F7063
:100B5000862F90E0A0E0B0E0022E04C0880F991F1D
:100B6000AA1FBB1F0A94D2F7D4FF10C04FE050E079
:100B700060E070E004C0440F551F661F771F2A9580
:100B8000D2F7409550956095709503C040E050E0D5
:100B9000BA01C695C695C3708A019B01082B192B13
:100BA0002A2B3B2BC901B801C23049F058F4C1309F
:100BB00019F00E94160881C00E9404087EC00E949D
:100BC00028087BC00E94770778C0CF70112339F0C6
:100BD0008C2F0E949D078D2F0E9451046EC08D2F77
:100BE0000E9458048C2F0E94BE0767C0D23F21F19B
:100BF00028F4D03F41F0D13FC1F043C0D33F19F1B9
:100C0000D43F79F03EC0112341F0053008F051C0C7
:100C10008C2F8F710E94E3074CC0063008F049C04A
:100C2000F7CF8091070382FF18C0112339F08C2F72
:100C30008F710E949D073DC01123C9F38C2F8F71C6
:100C40000E94BE0736C0112329F08C2F8F710E949D
:100C500088072FC00E9483072CC0112349F0CF7151
:100C60008C2F0E949D0763E08C2F0E94BF0C21C037
:100C700081E00E94DA0C0230E0F082E00E94DA0C9F
:100C800018C0112331F0002391F28D2F0E94300300
:100C900010C0002399F2D93349F41FEF27EE33E057
:100CA000115020403040E1F700C000008D2F0E941D
:100CB000D20388EF8C0D843020F40E9483140E94AC
:100CC000C502DD20C9F00E942D0C80FD15C0F70182
:100CD00012820E94270C0E949D07C7010E949D0658
:100CE0000E94270CDF91CF911F910F91FF90EF9001
:100CF000DF90CF900C94BE07DF91CF911F910F91A1
:100D0000FF90EF90DF90CF9008950F931F93CF93B4
:100D1000DF93EC01688179818A810E94DF088C0170
:100D20000E943A080E942B07B801CE010E945F047E
:100D3000DF91CF911F910F910895CF93DF93EC0135
:100D4000988189812B813C81232B31F08F3F31F4B5
:100D500081E09F3F19F403C081E001C080E080FD85
:100D60001DC0CE010E946302811110C00E94310C8F
:100D70008823A1F08A81882389F08091070382FD6E
:100D80000DC082E0DF91CF910C94DA0CCE010E946D
:100D90008506CE01DF91CF910C944402DF91CF9173
:100DA000089580E090E00E94A91480E090E00E9405
:100DB000BF140E94580C0C947A0C809102019091FF
:100DC00003010E9481150C94D1060E94480C0C94DA
:100DD000DD0692959F70963079F010F4925001C024
:100DE0009A50923068F4803F69F018F4883E40F4DD
:100DF00009C0843F29F406C0883E20F0813F11F0ED
:100E000080E0089581E00895FC01808191810E9435
:100E1000D4080E94E9060895CF93DF9300D000D054
:100E20001F92CDB7DEB70F900F900F900F900F90DD
:100E3000DF91CF910895CF93DF9300D000D000D001
:100E4000CDB7DEB726960FB6F894DEBF0FBECDBF86
:100E5000DF91CF910895089508950C942C070C9478
:100E60002D070E942F0760932B0270932C02809312
:100E70002D0290932E020C94D1060C9431070F93FF
:100E80001F9300912B0210912C0220912D02309182
:100E90002E02602B712B822B932B1F910F910C94A0
:100EA00031070F931F9300912B0210912C02209178
:100EB0002D0230912E0260237123822393231F91F0
:100EC0000F910C9431070F931F9300912B021091F7
:100ED0002C0220912D0230912E026027712782274B
:100EE00093271F910F910C9431070C942C070E94AB
:100EF00075076093270270932802809329029093CC
:100F00002A020C94D10660E070E0CB010C947707C4
:100F10000F931F9341E050E060E070E08A019B0175
:100F200004C0000F111F221F331F8A95D2F7C90179
:100F3000B8011F910F910C9477070F931F9341E015
:100F400050E060E070E004C0440F551F661F771F3B
:100F50008A95D2F78091270290912802A0912902C8
:100F6000B0912A028A019B01082B192B2A2B3B2BBB
:100F7000C901B8011F910F910C9477070F931F932C
:100F800041E050E060E070E004C0440F551F661F70
:100F9000771F8A95D2F7409550956095709580910E
:100FA000270290912802A0912902B0912A028A0179
:100FB0009B01082319232A233B23C901B8011F9150
:100FC0000F910C9477070F931F9341E050E060E07E
:100FD00070E004C0440F551F661F771F8A95D2F733
:100FE0008091270290912802A0912902B0912A02B3
:100FF0008A019B01082719272A273B27C901B80125
:101000001F910F910C9477070F931F930091270264
:10101000109128022091290230912A02602B712B15
:10102000822B932B1F910F910C9477070F931F9393
:1010300000912702109128022091290230912A0262
:1010400060237123822393231F910F910C947707C0
:101050000F931F93009127021091280220912902DB
:1010600030912A0260277127822793271F910F91C1
:101070000C94770708952FE0929F800D1124E82F9C
:10108000E695E695E695877051E001C0550F8A9583
:10109000EAF785E0E89FF0011124EA56FE4F20E0D0
:1010A00030E070E04081CB01022E02C0969587951A
:1010B0000A94E2F7817081958427852384278193A0
:1010C0002F5F3F4F2530310569F708952FE0929F3C
:1010D000800D1124682F669566956695982F9770F8
:1010E00085E0689FB001112440E050E080E0FB0102
:1010F000E40FF51FEA56FE4F208130E0092E02C0B2
:10110000369527950A94E2F721703327042E01C003
:10111000220F0A94EAF7822B4F5F5F4F453051054B
:1011200031F70895BF92CF92DF92EF92FF920F9323
:101130001F93CF93DF938C01C0902702D090280299
:10114000E0902902F0902A0280912B0290912C02CB
:10115000A0912D02B0912E02C82AD92AEA2AFB2A90
:10116000CFE1D0E0D701C6010C2E04C0B695A795FB
:10117000979587950A94D2F780FD04C0219790F740
:10118000B12C07C0BC2EB8018C2F0E94C30F019751
:10119000A9F38B2DDF91CF911F910F91FF90EF90CD
:1011A000DF90CF90BF900895CF93DF93EC010E9422
:1011B0009208BE010E94C30FDF91CF9108951F9343
:1011C000CF93DF93EB0190919501992321F0CB010F
:1011D0000E94D40813C0882349F0CB010E949208D2
:1011E000182F682FCE010E943B0804C0CB010E943B
:1011F0006608182FBE01812F0E94C30FDF91CF9187
:101200001F9108951F93CF93DF93C0912F0216E093
:1012100080913002C81799F0D0E01C9FF0011D9F0B
:10122000F00D1124EF5CFD4F40815181628173818B
:10123000848195810E941B072196C770E9CFDF91B9
:10124000CF911F9108954091610250916202609187
:1012500063027091640280916502909166020C9421
:101260001B07EF92FF920F931F93CF93DF93809111
:10127000660282958F7009F065C0809163028823B1
:1012800009F460C080912F02F09030021091610249
:1012900000916202609164027091650291E01F3FCB
:1012A00009F090E0C0910001D0910101292F96E052
:1012B000E92E8F1509F446C06115710521F00F3F25
:1012C00021F030E003C031E001C0322F90E030FD6A
:1012D00036C0E89EF001E99EF00D1124DF01AF5CFD
:1012E000BD4F11963C911197301329C03C91311399
:1012F00026C012963C911297311121C013964D9140
:101300005C911497461B570B4C175D07C0F48091F6
:1013100066028F70806180936602EA5CFD4F808177
:101320008F708061808381E692E00E949D06DF914C
:10133000CF911F910F91FF90EF900C9402090196AD
:101340008770B7CFDF91CF911F910F91FF90EF90F2
:1013500008959F92AF92BF92CF92DF92EF92FF9249
:101360000F931F93CF93DF93CDB7DEB761970FB67F
:10137000F894DEBF0FBECDBF8C0185E0F801DE0121
:101380001D9601900D928A95E1F7D8011296EC9086
:1013900090916102E09162022091640230916502B5
:1013A0002115310531F0EF3F31F481E09F3F19F411
:1013B00003C081E001C080E0B82FB1709B2E80FD9A
:1013C00047C1D8014C9111965C9111971396AD903D
:1013D000BC90149781E6C82E82E0D82EF09063026C
:1013E000B501621B730B2091000130910101FF20B8
:1013F00009F4D9C0809166026217730708F095C09E
:10140000282F207F09F052C05E1313C0491311C06A
:10141000FE2CE1100EC08F708061809366020E94E6
:101420002309C6010E949D0680916602F80185830A
:101430004DC1AB2831F05F3F31F481E04F3F19F4EB
:1014400003C081E001C080E080FD03C081E08E2503
:1014500002C080E090E0F82FF170FF2E80FF1CC0EA
:1014600080912F022091300236E0821709F40BC1DF
:1014700090E0389FF001399FF00D1124EF5CFD4F93
:101480006181561306C06081461303C06281E61273
:1014900003C001968770E9CFFE2CEE2009F416C137
:1014A0008091660281608093660254C05E1306C01C
:1014B000491304C0E11002C0F80199C0C8010E949C
:1014C0000407882361F1EE2051F120916602822FFA
:1014D00082958F7090E0029774F0809161029091F4
:1014E000620298878F831986BB86AA862C87CE01D5
:1014F00007960E949D0686E0F801A1E6B2E0019001
:101500000D928A95E1F70E9431090E9423090AC0D1
:101510005E1711F1C8010E94040781112CC0C80197
:101520000E949D06FF24F394D1C0282F207F81F7CD
:101530007A2DB98AA88A6E2D89890E940C0781E6C6
:1015400092E00E949D0686E0D6011D928A95E9F7F9
:101550000E942309F12CBAC04913DCCFE110DACF85
:10156000F8018583C8010E949D0686E0D6011D9280
:101570008A95E9F7ABC0EE2091F220916602822FA6
:1015800082958F7090E002970CF4B5CF8091610244
:10159000909162029A8389831B82BD82AC822E83E2
:1015A000CE010196A6CF6217730708F044C0FE2C47
:1015B000EE2009F4B4CF5E1330C049132EC0209141
:1015C000660220FD21C0822F82958F70482F50E047
:1015D00041155105C9F0F80125834F30510541F0FF
:1015E0008F5F982F9295907F822F8F70892B8583A4
:1015F000C8010E949D0686E0F801A1E6B2E00190D4
:101600000D928A95E1F73CC086E0F801A1E6B2E0D0
:1016100001900D928A95E1F759C0C8010E94040714
:10162000811169CF80916602816080936602C80152
:101630000E949D064BC07A2DB98AA88A6E2D898991
:101640000E940C0786E0D6011D928A95E9F718C022
:10165000EE2009F464CFC8010E940407F82E882305
:1016600009F45DCF86E0F801A1E6B2E001900D92A9
:101670008A95E1F781E692E00E942A030E943109EF
:101680000E94230923C04D875E878D859E850E9419
:10169000D408292F22952F70223028F49F7039F01A
:1016A000811105C00BC0243028F49F7049F4805E7E
:1016B000883020F0C8010E949D069F2CF92C06C09E
:1016C000D80115969C91907F91F7F8CF8F2D619658
:1016D0000FB6F894DEBF0FBECDBFDF91CF911F9143
:1016E0000F91FF90EF90DF90CF90BF90AF909F90C1
:1016F00008951F93CF93DF93CDB7DEB72C970FB626
:10170000F894DEBF0FBECDBF4F83588769877A87B5
:101710008B879C87CE0107960E94A9098823D1F068
:101720009F8188852A853B85232B31F08F3F31F4BB
:1017300081E09F3F19F403C081E001C080E080FD9B
:1017400047C04F81588569857A858B859C850E9425
:101750001B073EC086E0FE013796DE011196019020
:101760000D928A95E1F7FF81E8856A857B85611591
:10177000710531F0EF3F31F481E0FF3F19F403C010
:1017800081E001C080E080FD23C02091300230E084
:10179000C90101968770992740912F0250E0841764
:1017A0009507F1F1F983EA837D836C8396E0929F3C
:1017B000D001939FB00D1124AF5CBD4FFE01319657
:1017C00001900D929A95E1F7809330020E940209F0
:1017D00016E080912F0290913002891771F1189FC5
:1017E000C00111248F5C9D4F0E94A909882329F113
:1017F000E0912F021E9FF0011124EF5CFD4F40810C
:10180000518162817381848195810E941B0780913F
:101810002F0290E001968770992780932F02D9CFED
:101820000E94E5061092300210922F02E1E6F2E0EB
:1018300086E0DF011D928A95E9F72C960FB6F894A1
:10184000DEBF0FBECDBFDF91CF911F910895809174
:101850008702859585958595089580918702877083
:10186000089590918702977081E009F480E00895CF
:101870008091AA0208959091AA02892B8093AA02CE
:10188000089580959091AA0289238093AA020895D1
:101890001092AA0208959091A902892B8093A9021F
:1018A000089580959091A90289238093A9020895B3
:1018B0001092A902089580918802089508950C94C9
:1018C0005E0C0C945F0C9091070392FD08C0909100
:1018D0008802981721F0809388020C94610C089577
:1018E00080918802882329F01092880280E00C946D
:1018F000610C0895CF93DF93E0910201F091030111
:101900008091AA028083E0910201F091030190810D
:101910008091A902892B808380918802882381F09D
:10192000E0910201F09103019081892B80838091E5
:101930000201909103010E94D51481110E94700C44
:10194000C0910201D091030140E250E067E672E0ED
:10195000CE010E947F1D892B69F080E2FE01A7E67F
:10196000B2E001900D928A95E1F7CE01DF91CF911F
:101970000C948F14DF91CF9108950C945E0C90918C
:10198000070392FD10C098E0899F90011124262B37
:10199000209387020E949D078091870285958595F7
:1019A00085950C94BD0C0C949D071092870280E0E5
:1019B0000C94BD0C2091870280958223809387022E
:1019C000982F977099F430E0482F082E000C550B93
:1019D0002417350759F09091070392FD07C08595AC
:1019E000859585950E94BE070C94D50C089590911D
:1019F000070392FB222720F9281769F080FB92F950
:101A00009093070380910603909107030E943F0D76
:101A100082E00C94DA0C08958091070382FB8827FA
:101A200080F991E089270C94F70C81E00C94F70C75
:101A300080E00C94F70C80E090E00E94941D21E07F
:101A4000893E9E4F09F020E0822F089582E090E0C9
:101A50000C948C1D83E090E00C948C1DCF9384E05B
:101A600090E00E948C1DC82F82E290E00E948C1DA5
:101A70002C2F30E0A901582BCA01CF910895CF93A4
:101A8000C92F682F84E090E00E949A1D6C2F82E29B
:101A900090E0CF910C949A1DAB01BC018FE090E0D7
:101AA0000C94AC1DAB01BC0183E190E00C94AC1D27
:101AB00060E070E0CB010C94520D60E070E0CB016F
:101AC0000E944C0D0C94580D69EE7EEF80E090E082
:101AD0000E94B81D60E082E090E00E949A1D60E0E4
:101AE00083E090E00E949A1D10922B0210922C022B
:101AF00010922D0210922E0260E084E090E00E948D
:101B00009A1D60E082E290E00E949A1D60E085E00C
:101B100090E00E949A1D60E086E090E00E949A1D8D
:101B20006FEF87E090E00E949A1D40E050E0BA011C
:101B300088E090E00E94AC1D60E08DE090E00E94A3
:101B40009A1D40E050E0BA0188E190E00E94AC1D8F
:101B500060E087E190E00E949A1D40E050E0BA0109
:101B60008CE190E00E94AC1D60E070E080E290E0CB
:101B70000E94B81D40E050E0BA0188E190E00E9468
:101B8000AC1D0C945D0D0C94640D682F8EE090E0FC
:101B90000C949A1D0E943B166093CD027093CE0266
:101BA0008093CF029093D0026093C9027093CA02CF
:101BB0008093CB029093CC02089585B7806885BF4F
:101BC00085B7806885BF089581E008950C94E40D81
:101BD00008950C94E80D0C94E80D0C94EB0D0C9406
:101BE000E80D0C94EF0D0C94E80D0E94DD0D8FE9CB
:101BF00090E10E9479140E94F30D0C94F10D0E9463
:101C0000E90D0C94E80D0E94A2100C94C4020E94ED
:101C100026160E9487110E94030E0C94ED0D5F9210
:101C20006F927F928F929F92AF92BF92CF92DF92EC
:101C3000EF92FF920F931F93CF93DF93CDB7DEB751
:101C40002A970FB6F894DEBF0FBECDBF0E949C113D
:101C5000C82E81110E94CA0D3BEA832E32E0932EDA
:101C600000E010E0502E802F0E94C6105C01F401AD
:101C7000619071904F016826792661147104B1F466
:101C80000F5F1F4F0F30110569F78FEF89838A832C
:101C90001B820E942F168160782F9D838C8349813F
:101CA0005A816B818D810E94E0023AC08091D102FD
:101CB00081FD0E94CF10D12CEE24E394F12CC301BE
:101CC0008E219F21892B29F10E94E60D8823A9F0FE
:101CD000DE825F82AE20BF2081E0AB2809F480E085
:101CE00088870E942F168160782F9A8789874E8176
:101CF0005F8168858A850E94E002000F111FF8014C
:101D0000E555FD4F80819181E826F926F182E08238
:101D100007C0D394EE0CFF1CFFE0DF12D0CFB0CF92
:101D200081E0C11001C080E02A960FB6F894DEBFB2
:101D30000FBECDBFDF91CF911F910F91FF90EF901C
:101D4000DF90CF90BF90AF909F908F907F906F90DB
:101D50005F9008950E940F0E0C94D502CF93DF93ED
:101D60000E94C80FEC01811522E59207E8F5811564
:101D700031E5930708F0B6C0883E910528F5803E0E
:101D8000910508F0E9C0883A910570F4853A91050B
:101D900008F07AC08130910509F473C008F4D9C005
:101DA000049708F0D9C0D5C08F3B910508F0D1C089
:101DB000C85AD0E0CC0FDD1FCE5BDE4F0990D88132
:101DC000C02DCE019464C9C0811540E5940708F088
:101DD00069C0811550E4950708F060C09A95811597
:101DE0009F4108F4B9C0B5C0811536E5930728F5C1
:101DF000811545E5940708F092C0811554E59507D3
:101E000008F087C0AC0143705527282F26952695EA
:101E1000C115D34508F06CC081E090E002C0880F86
:101E2000991F4A95E2F740E2249F90011124EC01AA
:101E3000C22BD32BCE019C6890C081152AE5920756
:101E400080F4811539E5930708F072C0811548E5E3
:101E5000940708F47EC0D82FCC27CE01806F906AFB
:101E60007CC090568115904208F073C08D2F8F7101
:101E70000E945C10DD27D0628F71AE01582BCA0121
:101E80006CC081E090E069C0C55AD0E0C059DE4F17
:101E90008881C82FD0E0CE0190645FC0DF70CE0192
:101EA000906A5BC074E0969587957A95E1F7282F44
:101EB00023703C2F337081E090E002C0880F991F9F
:101EC0003A95E2F79C68AC01522B9A019C2F9F70C7
:101ED0009695969550E2959FE0011124C9018C2BAF
:101EE0009D2B3BC0D82FCC27CE01816F906A35C087
:101EF00081E090E002C0880F991F4A95E2F750E216
:101F0000259F90011124EC01C22BD32BCE019A689E
:101F100024C0D82FCC27CE01846F906A1EC00E94A7
:101F20005C108F7190E0D82FCC27CE01906215C045
:101F30008F700E945C1094E0D695C7959A95E1F752
:101F4000CF70D0E0DC2FCC27D0699E01282BC901AF
:101F500004C080E090E001C0CE01DF91CF910895F0
:101F600021EE829FC0011124FC012FE0729FE00D41
:101F7000F11D1124E60FF11DEE0FFF1FEC53FF4F73
:101F80008591949108950E94B00F0E94AE0E08951D
:101F90008238910569F1B0F48133910509F46DC07F
:101FA00048F48932910509F463C08A32910509F435
:101FB00069C008958533910509F455C089339105A9
:101FC000B9F00895833E910569F138F4803E91059A
:101FD000B1F0823E910509F10895863E9105A9F17F
:101FE000873E9105B9F1843E910509F064C023C094
:101FF0002091060320FD4FC021FD4DC00895809122
:10200000060380FD44C08091070380FF44C0809197
:10201000060384FD42C083EE4DC08091060382FF1B
:1020200038C0F5CF8091060382FD33C0809107034D
:1020300080FD31C0ECCF8091070381FF32C08091D9
:10204000060384FD2AC087EE35C08091060383FF16
:1020500026C0F5CF8091060383FD21C08091070340
:1020600081FD1FC0ECCF8091060385FD1CC01DC003
:102070008091060385FD19C016C08091060386FD78
:1020800016C017C08091060386FD13C010C089E3F7
:1020900011C082EE0FC080EE0DC080E00BC086EE56
:1020A00009C084EE07C089E205C085E303C08AE267
:1020B00001C081E390E008959091060392FF0DC066
:1020C000282F2871283019F4877F846006C0282FB4
:1020D0002471243011F48B7F886093FF0DC0282F6A
:1020E0002871283119F4877E846106C0282F247155
:1020F000243111F48B7E88612091070320FF0DC0ED
:10210000382F3871383019F4877F816006C0382F36
:102110003171313011F48E7F886021FF0DC0282F7E
:102120002871283119F4877E816106C0282F21711A
:10213000213111F48E7E886194FD877E089580E0C0
:10214000089508950E941B0D811102C00E94C30DC5
:102150000E94260D8093D1020E942E0D90930703BA
:10216000809306030E94A1100E942A0D682F70E040
:1021700080E090E00E943D07609127027091280264
:102180008091290290912A020C947507E82FF0E0C3
:10219000EE0FFF1FEA5DFC4F808191810895089545
:1021A00080EA8A95F1F7089500C008950C94D01044
:1021B00008950C94D8100C94D9100C94D8100C9449
:1021C000DD10F894E82FE295EF70F0E031A1282FB0
:1021D0002F7081E090E001C0880F2A95EAF7982FD0
:1021E0009095932391A392A1892B82A3789408952B
:1021F0000F931F93CF93DF93C2E8D1E089918F3F74
:1022000011F00E94E11081E0C139D807B9F7C3E7A6
:10221000D1E002E811E089918F3F11F00E94E110B6
:102220000C171D07C1F7DF91CF911F910F910895F2
:10223000BF92CF92DF92EF92FF920F931F93CF93B3
:10224000DF938C01C62FD0E0CE018E579E4F6C01DC
:10225000FC0190819F3F09F450C0B62EF894E92FFD
:10226000E295EF70F0E081A19F7021E030E001C0C5
:10227000220F9A95EAF7822B81A382A12095282329
:1022800022A378940E94D410E3E7F1E042E851E001
:1022900021E030E0E12CF12C61916F3F89F0A62F15
:1022A000A295AF70B0E090968C9190E06F7002C0F4
:1022B000959587956A95E2F780FD02C0C90102C035
:1022C00080E090E0E82AF92A220F331F4E175F07BB
:1022D00019F7F60180818F3F11F00E94E11061E053
:1022E000E114F10409F460E08B2D0E94D610CC0FAC
:1022F000DD1FC00FD11FF982E882DF91CF911F91BE
:102300000F91FF90EF90DF90CF90BF9008950E94C3
:10231000F8108EE1E6E2F3E0DF01982F1D929A9526
:10232000E9F7E8E0F3E0DF011D928A95E9F78FE035
:102330000E94E7110C944F02FF920F931F93CF93CB
:10234000DF93CDB7DEB76E970FB6F894DEBF0FBE42
:10235000CDBF8E010F5F1F4F8EE1F80111928A955C
:10236000E9F7F12C6F2DC8010E941811F394FFE0DA
:10237000FF12F8CF4EE150E0B80188E093E00E94F0
:102380007F1DFF24F394009709F4F12C892B41F071
:102390008EE1F801A8E0B3E001900D928A95E1F793
:1023A0002F2D4FE066E273E088E093E00E94E81191
:1023B0000E9451028F2D6E960FB6F894DEBF0FBEAD
:1023C000CDBFDF91CF911F910F91FF900895089598
:1023D000FF920F931F93CF93DF93F82E092F162FA1
:1023E000D72FC42F222349F081E08093D4020E948A
:1023F0002F169093D3028093D2028091D402882327
:10240000D9F08091D2029091D3020E94471605978D
:1024100098F0EF2DF02FA12FBD2F80E090E04C2FF2
:1024200050E08417950734F4219131912D933D9319
:102430000196F7CF1092D402DF91CF911F910F91A7
:10244000FF9008950E9435180E94070E0C944118C1
:102450000E9445180E94AA0E0C945F180E94CD1588
:102460000E941C180E94F50D0E9422120E94281240
:102470000E94FF0DFBCFCF93DF93EC01FB01828124
:10248000882309F43CC1C430FDE5DF0760F4CB3F8D
:102490009CE5D90788F49E0122503C452431310542
:1024A00008F02EC109C0C236EDE5DE0729F0C63AB4
:1024B000FDE5DF0709F024C10E942E0D909307036C
:1024C00080930603C1318CE5D80709F4C6C008F033
:1024D00042C0C930ECE5DE0709F49BC000F5C53009
:1024E0008CE5D80709F485C078F4C330ECE5DE0745
:1024F00009F478C008F07AC0C230DC4509F0F5C0B4
:10250000809106038160EFC0C7309CE5D90709F4CC
:1025100078C008F07AC0809106038061E4C0CD30B5
:10252000FCE5DF0709F487C058F4CB309CE5D907F8
:1025300009F479C008F07BC08091060388606FC001
:10254000CF30FCE5DF0709F480C008F082C080913D
:102550000603877FC8C0CE3F9CE5D90709F471C048
:1025600000F5C531FCE5DF0709F485C068F4C33127
:102570009CE5D90709F475C008F095C00E94E506EE
:10258000809106038F77AFC0CC3FFCE5DF07A9F150
:1025900008F054C0CB3FDC4509F0A7C08091070389
:1025A00040C0C230EDE5DE0709F489C058F4C1151A
:1025B0008DE5D80709F45AC008F069C08091070377
:1025C00082602FC0C236EDE5DE0709F47CC0C63A52
:1025D000FDE5DF0709F481C0C330DD4509F085C0A2
:1025E00080E06EC08091060382607DC0809106030A
:1025F00016C080910603886076C0809107038260D0
:102600004FC08091060380626EC080910603806493
:102610006AC00E94E50680910603806864C08460F9
:1026200062C081603DC0809106038E7F5CC0809156
:1026300006038D7F58C08091060316C08091070362
:1026400018C0809107038D7F2BC0809106038F7E79
:102650004AC0809106038F7D46C0809106038F7B20
:1026600042C080910603877F8B7F3DC08091070326
:102670008D7F8E7F15C08091060382FB222720F973
:1026800091E0922790FB82F990FB83F92CC0809116
:102690000703982F909591708E7F892B90FB81F97D
:1026A0008093070322C00E94E5068091060387FB02
:1026B000222720F991E0922790FB87F914C081E04E
:1026C0000E94C50D12C08091060384FB222720F9C9
:1026D00091E0922790FB84F906C080910603982F21
:1026E000909590FB80F9809306038091060390916A
:1026F00007030E943F0D0E94E50680E001C081E0D3
:10270000DF91CF910895CF93DF9386319C4541F5BA
:10271000EB010E94380C982F8A81209102013091A0
:102720000301882379F09A7A81E009F480E08093AC
:10273000D502911102C069E201C065E3C9010E949E
:102740006B150AC08091D502811102C069E201C0F7
:1027500065E3C9010E9476150E947A0C80E001C0F1
:1027600081E0DF91CF9108950F931F93CF93DF9373
:10277000C42FD22FFC0182818823C9F04093D80254
:102780000E942F169093D7028093D60280E28C0F7E
:10279000883008F057C0C77081E001C0880FCA9523
:1027A000EAF7DF91CF911F910F910C945104809122
:1027B000D802481330C08091D6029091D7020E946F
:1027C0004716883C910538F510E21D0FCD17B9F07A
:1027D00080E28C0F883040F4C77081E001C0880F20
:1027E000CA95EAF70E945804183028F581E09D2F19
:1027F000977001C0880F9A95EAF70E945104802FC4
:102800000E9448041830F0F4D77081E001C0880FAE
:10281000DA95EAF70AC080E28C0F883098F4C77026
:1028200081E001C0880FCA95EAF7DF91CF911F912F
:102830000F910C945804802FDF91CF911F910F912D
:102840000C944804DF91CF911F910F9108950F933D
:102850009C01CB01243F4CE5340731F188F4293D3C
:10286000FCE53F07D9F02A3D4CE5340779F1283DD6
:102870003C45A9F506E221EE41EE68ED7CE52BC072
:10288000263FFCE53F07E1F0A8F0273F3C4539F53E
:1028900007E225EE46EE67EF7CE51DC007E225EE78
:1028A00045EE69ED7CE517C006E221EE40EE64EFEF
:1028B0007CE511C007E225EE44EE65EF7CE50BC038
:1028C00006E221EE42EE66EF7CE505C008E221E07B
:1028D00045EE6AED7CE50E94B41380E008C0FC017F
:1028E0008281882319F01092D80201C081E00F91F3
:1028F0000895909393018093920108959093DE023E
:102900008093DD020895E091DD02F091DE023097C0
:1029100021F00190F081E02D099480E00895E0918C
:10292000DD02F091DE02309799F020911001222310
:1029300059F02091060327FF07C0DC012C91119666
:102940002C93119726E02C930280F381E02D0994BB
:1029500008952091DB023091DC022817390771F0CD
:102960009093DC028093DB02E091DD02F091DE02C5
:10297000309721F00680F781E02D09940895209189
:10298000D9023091DA022817390771F09093DA02F0
:102990008093D902E091DD02F091DE02309721F0C0
:1029A0000084F185E02D09940895FC013296809110
:1029B0001001882331F08091060387FF02C09EE159
:1029C00001C096E080E0915028F021912223D9F3B4
:1029D0008F5FF9CF0895662351F1209110012223D2
:1029E000E9F02091060327FF19C0462F469546952A
:1029F00046954E31E0F4677021E030E002C0220FCE
:102A0000331F6A95E2F7FC01E40FF11D828190E02B
:102A10002823392381E0232B69F409C0FC01329675
:102A200008962191621729F0E817F907D1F780E09D
:102A3000089581E008959C01FC0132969FEF80E0AB
:102A40004191461789F09F3F19F4411101C0982F19
:102A50008F5F8630A9F79F3F39F0F901E90FF11D2B
:102A600097FDFA956283089508959C012A5F3F4F70
:102A7000FC014281461301C012820196821793071E
:102A8000B9F70895262F2695269526952E3168F4B8
:102A9000FC01E20FF11D677021E030E001C0220F60
:102AA0006A95EAF78281282B22830895262F26959E
:102AB000269526952E3170F4FC01E20FF11D67700A
:102AC00021E030E001C0220F6A95EAF7209582816B
:102AD00028232283089520911001222329F0209198
:102AE000060327FD0C9442150C941B152091100130
:102AF000222329F02091060327FD0C9456150C94EF
:102B0000351520911001FC013296222331F080917D
:102B1000060387FF02C08EE101C086E0DF011D923F
:102B20008A95E9F7089508950C94931583E08093AE
:102B3000DF020C949415811102C081E001C082E093
:102B40008093DF020C9494150C949B1581E0809384
:102B5000DF020C9494150C94A61508950C94AD15F1
:102B60000C94AE150C94AD150C94AD150C94AD15DC
:102B7000CF930E94B4150E949C110E94B215C0E030
:102B80008C2F0E94C610892B29F4CF5FCF30C1F75C
:102B900080E001C081E0CF91089508951F920F92C7
:102BA0000FB60F9211248F939F93AF93BF93809191
:102BB000E002811113C08091440390914503A091DC
:102BC0004603B09147034196A11DB11D8093440374
:102BD00090934503A0934603B0934703BF91AF91F1
:102BE0009F918F910F900FBE0F901F90189580911D
:102BF0004C03843031F10E94B5021092E00220E4CF
:102C000088E190E00FB6F894A895809360000FBE1D
:102C10002093600083B7817F846083BF83B7816026
:102C200083BF7894889583B78E7F83BF0FB6F8945F
:102C3000A895809160008861809360001092600088
:102C40000FBE08950E94E5060C94B90282E084BD8F
:102C500093E095BD9AEF97BD80936E0008952FB7CE
:102C6000F8948091440390914503A0914603B0915C
:102C700047032FBF08952FB7F894609144037091D4
:102C8000450380914603909147032FBF08959C010F
:102C90004FB7F8948091440390914503A091460367
:102CA000B09147034FBF821B930B089578941F92F6
:102CB0000F920FB60F9211248F939F93AF93BF93F0
:102CC0008091440390914503A0914603B09147033E
:102CD0000196A11DB11D8093440390934503A093D9
:102CE0004603B0934703BF91AF919F918F910F908F
:102CF0000FBE0F901F901895F89481E08093E0002C
:102D000080E28093D800E9ECF0E010828FE19EE44D
:102D10000197F1F700C000001DBA109268001CBCBA
:102D200010BE1FBA10927A0010926E0010926F00BF
:102D3000109270001092710010821092BC0011B8B5
:102D400014B817B81AB81DB810BA12B815B818B810
:102D50001BB81EB811BA0C9400FE089580910403AC
:102D600008950895CF93DF9320911001222339F025
:102D70002091060327FF03C060E222E002C068E062
:102D800021E02093E9002FEF3091E800215035FD3C
:102D900006C035ED3A95F1F700002111F5CF2091ED
:102DA000E80025FF1DC0EC0180911001811105C0D4
:102DB00040E050E068E070E003C070E040E050E0C8
:102DC000CE010E94D1188091E8008E778093E800B0
:102DD00080E2FE01A4EEB2E001900D928A95E1F747
:102DE000DF91CF9108958093E1027093E3026093A5
:102DF000E20280914C03843001F582E08093E90087
:102E00008FEF9091E800815095FD06C095ED9A9561
:102E1000F1F700008111F5CF8091E80085FF0DC02A
:102E200040E050E063E070E081EE92E00E94D11853
:102E30008091E8008E778093E8000895BC0184E0DB
:102E40000C94F316BC0183E00C94F3160895809162
:102E50004B03811109C00E945E1A0E94C01A809122
:102E6000E20084608093E200089510924B0308957D
:102E70000C94AB156091480381E0611101C080E0C2
:102E80000C94961590914C0381E0943009F080E009
:102E9000609148030C949B1542E061EC81E00E9434
:102EA000D71942E261EC82E00E94D71990914C035D
:102EB00081E0943009F080E0609148030C94A415FF
:102EC00080914E03833009F45FC030F4813071F09B
:102ED000823009F498C008958A3009F484C08B3098
:102EE00009F46AC0893009F0A6C020C080914D0362
:102EF000813A09F0A0C08091E800877F8093E800C4
:102F00008091510390915203892B21F460E284EE69
:102F100092E003C060E080E090E070E00E941C1945
:102F20008091E8008B778093E800089580914D03AD
:102F3000813209F080C08091510390915203029731
:102F400008F079C08091E800877F8093E800809145
:102F5000E80082FD05C080914C038111F8CF6BC061
:102F60008091F2009091F300029731F48091F1008A
:102F7000813011F0863021F48091F10080930403B8
:102F80008091E8008B7753C080914D03813A09F01E
:102F900052C08091510390915203892B09F04BC08C
:102FA0008091E800877F8093E8008091E80080FFAF
:102FB000FCCF8091100136C080914D038132D9F54C
:102FC0008091510390915203892BA9F58091E800DB
:102FD000877F8093E8000E940C1A80914F038093B2
:102FE00010010C94E50680914D03813221F580910A
:102FF000E800877F8093E8000E940C1A80915003BC
:1030000080930503089580914D03813AA1F4809146
:10301000E800877F8093E8008091E80080FFFCCF84
:10302000809105038093F1008091E8008E77809372
:10303000E8000C940C1A089584B7877F84BF0FB6FC
:10304000F894A89580916000886180936000109248
:1030500060000FBE90E080E80FB6F89480936100A6
:10306000909361000FBE0C94A6150E945E1A0E94F8
:10307000C01AE2EEF0E080818460808378940C9442
:103080005B1D84E091E00C947E1480914C038530AC
:10309000A9F480914C03853079F40E94F715809152
:1030A0004A038823B1F30E94B815882391F30E9444
:1030B000BB180E94E506EDCF0C94221608950895E2
:1030C0000C946218292F332723303105C9F060F49E
:1030D0002130310581F02230310509F044C08BE305
:1030E00090E02EEB32E043C021323105E1F0223294
:1030F000310549F138C082E190E029EF32E037C074
:1031000099278130910549F028F0029761F5E6E8AA
:10311000F2E005C0EAEBF2E002C0E0EAF2E08491FE
:1031200090E09F0124C06115710541F06130710587
:10313000D1F489E090E029EE32E019C089E090E016
:1031400020ED32E014C06115710541F06130710568
:1031500051F48DE690E02BE033E009C080E490E08C
:1031600028E733E004C080E090E020E030E0FA019E
:1031700031832083089584E189BD86E189BD09B446
:1031800000FEFDCF8091D8008F7D8093D800809184
:10319000E00082608093E0008091E00081FDFCCF40
:1031A0000895CF92DF92EF92FF920F931F93CF93E8
:1031B000DF93EC018B017A010E942B1A811133C03D
:1031C000E114F10439F0F70180819181081B190B9A
:1031D000C80FD91FC12CD12C0115110519F18091EF
:1031E000E80085FD16C08091E8008E778093E800A6
:1031F000E114F10449F0F70180819181C80ED91ED4
:10320000D182C08285E00FC00E942B1A882321F34F
:103210000AC089918093F10001501109FFEFCF1A84
:10322000DF0ADACF80E0DF91CF911F910F91FF90FD
:10323000EF90DF90CF900895209153033091540385
:103240002617370748F06115710539F42091E80019
:103250002E772093E80001C0B901FC0120E0611540
:10326000710569F180914C038823E1F18530E1F12A
:103270008091E80083FD3AC08091E80082FD2CC077
:103280008091E80080FFEBCF8091F2009091F300F5
:103290006115710551F08830910538F42191209322
:1032A000F100615071090196F3CF21E0089709F010
:1032B00020E08091E8008E778093E800D0CF211144
:1032C000D1CF0AC080914C03882361F0853061F032
:1032D0008091E80083FD0AC08091E80082FFF2CF70
:1032E00080E0089582E0089583E0089581E00895E4
:1032F00020915303309154032617370748F0611586
:10330000710539F42091E8002E772093E80001C080
:10331000B901FC0120E06115710581F180914C0338
:10332000882309F43EC0853009F43DC08091E8004F
:1033300083FD3BC08091E80082FD2DC08091E800B4
:1033400080FFE9CF8091F2009091F3006115710543
:1033500059F08830910540F424912093F100319682
:10336000615071090196F2CF21E0089709F020E041
:103370008091E8008E778093E800CDCF2111CECFE9
:103380000AC080914C03882361F0853061F0809100
:10339000E80083FD0AC08091E80082FFF2CF80E060
:1033A000089582E0089583E0089581E00895982FBC
:1033B000973068F59093E900981739F07091EC0018
:1033C0002091ED005091F00003C0242F762F50E0A3
:1033D00021FD02C09F5FECCF3091EB003E7F309328
:1033E000EB003091ED003D7F3093ED003091EB002C
:1033F00031603093EB007093EC002093ED0050931C
:10340000F0002091EE0027FDE5CF80E008958F7059
:103410008093E90081E0089580914D0387FF11C0FA
:103420008091E80082FD05C080914C038111F8CFA6
:1034300011C08091E8008B770BC080914C038823EA
:1034400049F08091E80080FFF8CF8091E8008E7706
:103450008093E80008952091E4003091E50095E61E
:103460004091EC00842F817040FF23C08091E800E0
:1034700080FD1DC080914C03882399F0853099F020
:103480008091EB0085FD11C04091E4005091E50072
:103490002417350729F3915011F09A01E1CF84E008
:1034A000089582E0089583E0089581E0089580E022
:1034B00008954091E80042FFDDCF08950E94CF1AA1
:1034C0000E94D71AE0EEF0E0808181608083E8ED11
:1034D000F0E080818F77808319BCA7EDB0E08C91FC
:1034E0008E7F8C9380818F7E808310924B03089512
:1034F0000F931F93CF93DF930E94CF1A0E94D71A86
:10350000C8EDD0E088818F77888388818068888340
:1035100088818F7D8883E7EDF0E0808180688083FB
:1035200019BC10924C031092480310924A03109257
:10353000490300EE10E0F80180818B7F8083888151
:103540008160888342E060E080E00E94D719E1EE6C
:10355000F0E080818E7F8083E2EEF0E08081816008
:103560008083808188608083F80180818E7F808362
:10357000888180618883DF91CF911F910F91089599
:10358000E8EDF0E080818F7E8083E7EDF0E08081E0
:103590008160808381E080934B030C94781AE8ED7E
:1035A000F0E080818C7F80831092E2000895109279
:1035B000DA001092E10008951F920F920FB60F9259
:1035C00011240BB60F922F933F934F935F936F93FA
:1035D0007F938F939F93AF93BF93EF93FF938091CC
:1035E000E10082FF0BC08091E20082FF07C0809162
:1035F000E1008B7F8093E1000E945A1D8091DA00E8
:1036000080FF1FC08091D80080FF1BC08091DA002E
:103610008E7F8093DA008091D90080FF0DC084E115
:1036200089BD86E189BD09B400FEFDCF81E08093AC
:103630004C030E94271705C019BC10924C030E942E
:1036400035178091E10080FF19C08091E20080FF72
:1036500015C08091E2008E7F8093E2008091E200AD
:1036600080618093E2008091D80080628093D800CE
:1036700019BC85E080934C030E943A178091E100C9
:1036800084FF30C08091E20084FF2CC084E189BDBA
:1036900086E189BD09B400FEFDCF8091D8008F7D01
:1036A0008093D8008091E1008F7E8093E10080912B
:1036B000E2008F7E8093E2008091E200816080933F
:1036C000E20080914803882311F084E007C08091D4
:1036D000E30087FD02C081E001C083E080934C03DA
:1036E0000E9442178091E10083FF29C08091E2008F
:1036F00083FF25C08091E100877F8093E10082E015
:1037000080934C03109248038091E1008E7F809358
:10371000E1008091E2008E7F8093E2008091E200E0
:1037200080618093E20042E060E080E00E94D7196F
:103730008091F00088608093F0000E943817FF911C
:10374000EF91BF91AF919F918F917F916F915F9119
:103750004F913F912F910F900BBE0F900FBE0F9086
:103760001F9018951F920F920FB60F9211240BB64F
:103770000F922F933F934F935F936F937F938F930A
:103780009F93AF93BF93CF93DF93EF93FF93C0913A
:10379000E900CF708091EC00D82FD17080FDD0E887
:1037A0001092E9008091F000877F8093F000789478
:1037B0000E94FA1B1092E9008091F00088608093CB
:1037C000F000CD2BCF70C093E900FF91EF91DF9116
:1037D000CF91BF91AF919F918F917F916F915F91A9
:1037E0004F913F912F910F900BBE0F900FBE0F90F6
:1037F0001F9018951F93CF93DF93CDB7DEB7AA978D
:103800000FB6F894DEBF0FBECDBFEDE4F3E08091BC
:10381000F100819323E0E535F207C9F70E946017B4
:103820008091E80083FF2EC180914D0390914E035B
:10383000492F50E04A30510508F024C1FA01E85AF6
:10384000FF4F0C94761D803821F0823809F01AC1A0
:1038500008C08091490390914A03992389F08260BE
:103860000FC0809151038F70873008F00BC1809397
:10387000E9008091EB0085FB882780F91092E90030
:103880009091E800977F9093E8008093F100109268
:10389000F100D1C0282F2D7F09F0F4C0882319F042
:1038A000823061F0EFC080914F03813009F0EAC0AF
:1038B000933009F080E080934A032EC080914F033B
:1038C00081112AC0809151038F702FEF280F26306D
:1038D00008F0D8C08093E9002091EB0020FF1CC0C5
:1038E000933021F48091EB00806214C09091EB0042
:1038F00090619093EB0021E030E0A90102C0440FF9
:10390000551F8A95E2F74093EA001092EA008091F1
:10391000EB0088608093EB001092E9008091E80052
:10392000877F8093E8000E940C1AACC08111AAC066
:1039300010914F031F778091E3008078812B809353
:10394000E3008091E800877F8093E8000E940C1AD2
:103950008091E80080FFFCCF8091E3008068809335
:10396000E300111102C082E001C083E080934C03A8
:1039700089C08058823008F085C080914F039091B3
:1039800050038C3D53E0950779F583E08A838AE202
:1039900089834FB7F894DE01139620E03EE051E2B0
:1039A000E32FF0E050935700E49120FF03C0E2952D
:1039B000EF703F5FEF708E2F90E0EA3010F0C79607
:1039C00001C0C0968D939D932F5F243149F74FBF5F
:1039D0008091E800877F8093E8006AE270E0CE0182
:1039E00001960E941C1916C06091510370915203F8
:1039F000AE014F5F5F4F0E946018BC01892B09F434
:103A000041C09091E800977F9093E80089819A8166
:103A10000E9478198091E8008B778093E80032C08B
:103A2000803881F58091E800877F8093E80080915D
:103A300048038093F1008091E8008E7772CF811166
:103A400021C080914F039091500399270297D4F49D
:103A50008091E800877F8093E80080914F038093F6
:103A600048030E940C1A80914803811106C080917E
:103A7000E30087FD02C081E001C084E080934C0335
:103A80000E944C178091E80083FF0AC08091E800F3
:103A9000877F8093E8008091EB0080628093EB0049
:103AA000AA960FB6F894DEBF0FBECDBFDF91CF91BF
:103AB0001F9108950895CF9380914C038823A1F01E
:103AC000C091E900CF709091EC00892F817090FD3A
:103AD00080E8C82B1092E9008091E80083FD0E94E5
:103AE000FA1BCF70C093E900CF910895EE0FFF1F2E
:103AF0000024001C0BBE0790F691E02D0994FB01F9
:103B0000DC0104C08D910190801921F44150504096
:103B1000C8F7881B990B0895F999FECF92BD81BD16
:103B2000F89A992780B50895A8E1B0E042E050E006
:103B30000C94C01D262FF999FECF92BD81BDF89A35
:103B4000019700B4021639F01FBA20BD0FB6F894E1
:103B5000FA9AF99A0FBE08950396272F0E949B1D8B
:103B60000E949A1D252F0E949B1D242F0C949B1DA3
:103B70000196272F0E949B1D0C949A1DDC01CB01FE
:103B8000FC01F999FECF06C0F2BDE1BDF89A31966D
:103B900000B40D9241505040B8F70895F894FFCF0B
:103BA000C8008902AE16B216261722171E17B116C4
:103BB00001E200E900EA00B500B600B700CD0083DD
:103BC00001CC008A019201940121022302240225E2
:103BD00002260227022A02B300B4006F007000819F
:103BE0008283E200E900EA00B500B600B700CD002C
:103BF0008301CC008A019201940121022302240254
:103C00002502260227022A02B300B4006F007000CA
:103C10008182839697C0C13792939460343536F091
:103C2000C6C795F167F266F365F464F563F662F76B
:023C3000610031
:00000001FF
